:1006E0000000C8C80000C4C4C2C2C0C0C1C1CBCBD6
:1006F0000000C9C9C7C7C5C5C3C30909E0E00000F8
:10070000000000000000E4E400007151312100000D
:10071000000000007A5A735361417757322200F08B
:10072000000063437858644465453424332300F162
:10073000000020207656664674547252352500F229
:1007400000006E4E624268486747795936260000BD
:10075000000000006D4D6A4A7555372738280000A3
:1007600000002C3C6B4B69496F4F30003929000069
:1007700000002E3E2F2F6C4C3B2B70502D3D000067
:1007800000005C5F3A2A000040605E7E00000000CE
:10079000E1D200000D0D5B7B00005D7D00000000DC
:1007A0000000000000000000E3E300000808E2E2AF
:1007B0000000B1A15C7CB4A4B7A700000000000059
:1007C000B0A02E7FB2A2B500B6A6B8A81B1BD1D18F
:1007D000CACA2B2BB3A32D2D2A2AB9A9D0D0000029
:1007E000000000000000C6C6ABAB00000000000027
:1007F00000000000000000000000000000000000F9
:100000000BC052C170C107C006C005C004C070C19A
:1000100002C001C000C018950FED0DBF0FEF07BB68
:1000200003E401BB00E002BB02E005BF08E90AB936
:100030000CE009B933274BE074E588279927AA27F4
:10004000BB27CC2700E40BBF78949B7FEE2490FD68
:1000500003C092FFFCCF03C093FDC9F709C02E2D4A
:10006000743521F0783511F013D0EFCF2DD0EDCFCE
:10007000FC2CEBD008D091FF03C0FD2CE6D003D0C0
:100080009E7F9D7FE2CF9B7FEE2492FFFECF08955F
:100090005D9BFECF2CB908952F9326952695269526
:1000A000269520632A3310F007E0200F5D9BFECFDA
:1000B0002CB92F912F7020632A3310F007E0200F06
:1000C0005D9BFECF2CB9089580FD7DC0203E11F4CC
:1000D0008860A8C0213E11F48061A4C0203F11F4C3
:1000E0008160A0C0243171F483FD07C084FD9AC0F3
:1000F000A0FD98C0A16020E93FC0A3FD93C0A86007
:1001000023E93AC0213161F483FD05C0A2FD8AC014
:10011000A46022E931C0A5FD85C0A06225E92CC0FC
:10012000223129F4A1FD7EC0A26021E925C0293534
:1001300029F4A4FD77C0A06124E91EC0F3E0E0E744
:10014000E20F2227F21F8894EE1FFF1F0A2F027171
:1001500011F483FF01C0E160C895202D203B60F0C1
:100160002A3B50F4B1FF03C02F70206305C02F70ED
:10017000206A253A09F420E0213D19F484FD2AEA99
:1001800006C0203D21F40A2F097009F02AEAB2FFC7
:100190000BC0213420F02B3510F4206205C021362D
:1001A00018F02B3708F42F7D203051F0783511F0FE
:1001B000203808F46DDF203D18F0233D08F433D0DB
:1001C000877F8F7E2FC084FF03C0273759F526C055
:1001D000243151F483FD05C084FD24C0AE7F26E99F
:1001E00018C0A77F29E915C0213141F483FD03C060
:1001F000AB7F28E90EC0AF7D2BE90BC0223119F48B
:10020000AD7F27E906C0293519F4AF7E2AE901C080
:1002100005C0783511F0203808F43ADF8E7F877FEB
:100220008F7E00C00895203D11F401E007C0213DFC
:1002300011F402E003C0223D39F404E0B0279160DC
:1002400092600DEEC02EDB2E0895F894929894984B
:100250008A9A00E800000A95E9F78C9A8A9868E083
:1002600055271DD0F79410F08C9A02C08C985395A6
:1002700016D06A95B9F750FD02C08C9801C08C9ACF
:100280000ED08C980CD0849B03C00FEFF02EDDCFE6
:10029000829BFECF33274BE0882778940895829B7A
:1002A000FECF8299FECF08950FB60F921F939860EC
:1002B00082FD0BC04B3028F4433018F036958499FA
:1002C000306813E015BF84600AC012E015BF8B7F51
:1002D0004A9529F4E32E33274BE09460977F1F91D2
:1002E0000F900FBE18950FB60F920F900FBE189576
:1002F0000FB60F921F930F931CB1CC2309F04BC084
:100300001635A9F420E5C4DE20E5C2DE23E4C0DE14
:1003100021E4BEDE20E2BCDE26E5BADE21E3B8DE63
:100320002EE2B6DE20E3B4DE20E3B2DE50C01335A9
:1003300011F473E54CC0143511F474E548C0183558
:1003400011F478E544C01C3421F42B2F2063A0DE87
:100350003EC01B3461F42A2F2770206399DE2A2FB8
:100360002695269526952770206392DE30C012359B
:1003700031F491600FEFC02EAA27BB2728C0153497
:1003800011F4C86024C0113311F4C16020C01233CD
:10039000F1F4C2601CC0C3FF08C0916092600DEE12
:1003A000C02E1770D12ECC2712C0C0FF04C09160A0
:1003B000C12ECC270CC0C2FF05C091609260D12E27
:1003C000CC2705C0C1FF03C0C12EC46000C00F917F
:0803D0001F910F900FBE18955C
:00000001FF
